:020000040000FA
:1000000018308A00AD2E0000FF00030E8301A1000E
:100010000A08A0008A010408A2007708A300780853
:10002000A4007908A5007A08A6007B08A70083131E
:1000300083128C308400001C1F280C1832282208E0
:1000400084002308F7002408F8002508F900260892
:10005000FA002708FB0020088A00210E8300FF0E0B
:100060007F0E09008A110A1241280A108A100A110B
:10007000820700340034103430348A3400340034C1
:100080002D34061D452806114628061564000C105F
:100090008A110A121F28871087160530F700F70B00
:1000A0004F280000000000348C1A5828640054289F
:1000B0008C1E58281A088316CB008312981C6628B9
:1000C0001A088316CB0083121812181683164B08D1
:1000D000F800831200342908073C031D74280730F8
:1000E0000C1E70289900B32805308316B900390812
:1000F000063C0319B2283908053C031DAC282930F9
:10010000BB0083126F088316B800043083120C1EE4
:10011000872899006F080C1E8B2899008316BA0156
:1001200083126F0883163A020318A6283B0884003E
:100130000008BC0083120C1E9B28990083163B0804
:1001400084000008B806BB0ABA0A9028380883124F
:100150000C1EA82899008316831254207808831651
:10016000B9007728831200349030A9000130AA002A
:100170003930AB00831681138312861DC2280230EA
:10018000AC00C4280130AC000430EF006B20003418
:10019000D430840000080319DC280130F800F7018E
:1001A000F70BD028F80BCF283030F700F70BD62804
:1001B00000000000800BCD2800349130A9000230EF
:1001C000EF006B202A08F700F7080319F828013020
:1001D00077020319FE28023077020319042903303D
:1001E000770203190A290630770203191029172903
:1001F00005308316990022309800192902308316A1
:10020000990022309800192905308316990026306C
:100210009800192900308316990022309800192976
:10022000013083169900263098001929831283160D
:1002300019290230D4008312C8208A110A166528B1
:10024000F701F8018316510803105218F707F70C4D
:10025000F80CD218F707F70CF80C5219F707F70C3F
:10026000F80CD219F707F70CF80C521AF707F70C2D
:10027000F80CD21AF707F70CF80C521BF707F70C1B
:10028000F80CD21BF707F70CF80C831200349230ED
:10029000A9006F08413C031966290130AA008316A2
:1002A000B10131083F3C031C642902303107293E6B
:1002B00084003108D1000530D20083122021780853
:1002C00080008316B10A51299D2983128316B1013A
:1002D00031083F3C031C7F2901303107293E84004F
:1002E0000008B3003108D1000530D200831220216C
:1002F000780883163302031D7F29B10A6829310863
:100300003F3C031C85290130862900308312AA0056
:100310008316B10131083F3C031C9D29023031078F
:10032000293E84003108D1000530D20083122021FB
:10033000780880008316B10A8A2942308312EF00C0
:100340006B208A110A166D289530A9000508AA00AD
:100350000608AB000708AC00053083169F00831227
:100360001F083839C1389F000030F8001F08C7390E
:1003700078049F001E30F700F70BBC2900001F1502
:100380001F19C0291E08AD000830F8001F08C73922
:1003900078049F001E30F700F70BCC2900001F15D2
:1003A0001F19D0291E08AE000630EF006B20003464
:1003B0006F08073C031DEF292A0883168500831266
:1003C0002B088316860083122C088316870083125D
:1003D0002D0885002E0886002F088700A4218A1189
:1003E0000A1675282A088316B2002B30B300B10113
:1003F000023083126F028316310203182B2A32084F
:10040000B20AB4003308B30A84000008B500340807
:10041000831203178D008F0183160313350883128F
:1004200003178C0083168C130C15831203130B080F
:10043000F7008B138316031755308D00AA308D00FB
:100440008C148C18212A0C117708831203138B0447
:100450008316B10AF82907308312A9000130EF0092
:100460006B208A110A1685282A088316B2002B30C1
:10047000B30083122B08EF008316B10183126F08BB
:10048000831631020318582A3308B30A840032084D
:10049000B20AB500831203178D008F0183168C13E7
:1004A0000C1483120C08800083160313B10A3E2A31
:1004B000E3308312A9000230EF076B208A110A167D
:1004C0008D28E530A9000230AA00EF006B208A11C8
:1004D0000A169528E730A9004630AA000230EF003E
:1004E0006B208A110A169D28871200341930831652
:1004F000AA006330AB000330AC000230AD002E1018
:10050000AF0123303502FE3E03189D2A023E8312BE
:10051000A12A01308316A100A201A3010530A40085
:10052000A501A6019D2A8316A1016430A200A301A2
:10053000A401A501A6019D2A831683128A110A121D
:100540004B2B0A108A140A118207892A932A8316D0
:100550003308A0000130A100A201A3010530A400CE
:10056000A500A6010830A7000730A8004030A90068
:1005700020302002ED3E03184E2B133E8312612BD8
:1005800001308316AD002E10AF014E2B01308316C3
:10059000AD002E14AF014E2B8316AD012E10AF010E
:1005A0004E2B8316AD012E14AF014E2B0130831656
:1005B000A100A201A3016430A4000530A500A6019A
:1005C0000830A7000730A8002030A9002008223CEE
:1005D000031DEF2A0130AD002E14AF00F32AAD0148
:1005E0002E140130AF004E2B01308316A100A20162
:1005F000A3016430A4000530A500A6012030A700A7
:100600001F30A8004030A9002008253C031D0D2BF9
:100610000130AD002E14AF00112BAD012E140130AE
:10062000AF004E2B01308316A100A201A30164305C
:10063000A4000530A500A6014030A7003F30A80067
:100640004030A9002008263C031D2B2B0130AD00B3
:100650002E14AF002F2BAD012E140130AF004E2B06
:1006600002308316A100A201A3017830A4001E303D
:10067000A500A6011030A7000F30A8001030A90077
:100680000130AD002E140230AF004E2B831633081C
:10069000B5008312762A83164E2B83168317831692
:1006A000B40134083F3C031C5B2BA03034078400AA
:1006B0008001B40A512B7410831283138A110A1219
:1006C000A82B0A148A140A118207C62AC62AD62A17
:1006D000462B462BF42A122B302BC02AC62A4D2B30
:1006E000CC2AD12A4D2BD12AD12AD62AF42A122B50
:1006F00080308316870581308704D9308605061639
:10070000DB3085051B30850405158516861483129C
:10071000871107124B20742287140530F700F70B5E
:100720008F2B000000004B20742287140530F70047
:10073000F70B982B0000000020302802FF3E031822
:10074000A92B013EAC2B83163208B3008312A72AD3
:10075000A92B8A110A12BD2B0A148A140A118207C6
:10076000A32B2A088316B1003108E0398312A800B0
:1007700083163108B2008312782B0730A9000130AC
:10078000EF006B208A110A16A528831631108312F8
:100790002A080139003A0319D42B6F08023C031DC3
:1007A000D42B831631148312003083163118013094
:1007B000B200B30083124B2007110C3097000030B9
:1007C000F80004389200153083169200B30803191C
:1007D000F12B0B30831295001708CF399700F72BB8
:1007E00083160630831295001708CF3997004B20E7
:1007F00004308316B200AF30D4008312C8208316B1
:10080000B20BFB2B07308312A9000130EF006B20E5
:100810008A110A16AD280711970197014B2007305E
:10082000A9000130EF006B208A110A16B528831643
:10083000DF015F08033C031C2C2C0310DE0C0318A3
:10084000252C83120712272C83168312071687156F
:1008500087118316DF0A192C83120034871183163F
:10086000E30163080F3C031C452C0310E20CE10C70
:1008700003183E2C83120712402C8316831207168E
:10088000871587118316E30A312C64008312003424
:10089000D9308316DD00DE0183121724023083165F
:1008A0005D0784000008DE000E30E0005E08DF0017
:1008B0006008E2005E08E10083122E248316DE0148
:1008C000831217246E308316E200F830E1008312A1
:1008D0002E248316DE0183121724013083165D0750
:1008E00084000008DE000E30E0005E08DF006008D3
:1008F000E2005E08E10083122E248316DE018312DB
:1009000017246E308316E200F730E10083122E24A4
:100910008316DE018312172483165D088400000805
:10092000DE000E30E0005E08DF006008E2005E08D6
:10093000E10083122E248316DE01831217246E3009
:100940008316E200F630E10083122E240034D43006
:100950008400FC308005800C800C00080319B42C46
:10096000B22C0000800BB12C00348316DC013C302B
:10097000DB00DA010430D900831248240C308316DE
:10098000DE008312172483163708E2003608E100E0
:1009900083122E248316DE01831217248316E201AC
:1009A000E10183122E248316DE018312172483169D
:1009B00023082507B800D4008312C8208316240812
:1009C0002607B800D4008312A7248316E201E101B0
:1009D00083122E2400348316DC013C30DB00DA0164
:1009E0000530D900831248240C308316DE008312B0
:1009F000172483163708E2003608E10083122E24FC
:100A00008316DC013C30DB00DA010430D9008312AC
:100A100048240C308316DE0083121724831637080F
:100A2000E2003608E10083122E248316DE018312D1
:100A300017248316E201E10183122E248316DE01BE
:100A400083121724831623082507B800D4008312C5
:100A5000C820831624082607B800D4008312A724D0
:100A60008316E201E10183122E2400348316340838
:100A7000FD3E0318482D033E83124C2D0130831692
:100A8000B7008A30B6008312EB248316482D8316F4
:100A900083128A110A12002E0A148A100A1582077C
:100AA0003E2D472D3E2D83162F08FD3E0318032EA5
:100AB000033E8312072E83163208B4003408F70071
:100AC00001307702831203196D2DF7080319742D75
:100AD0000230770203198B2D912D8316B7018130D7
:100AE000B6008312B524922D8316B7018330B60069
:100AF0008312B52488308316B50035088F3C031C5B
:100B0000892DB7013508B6008312B5248316B50ABE
:100B10007D2D8312922D8316B7018030B60083128B
:100B2000B524922D8316032E83163208B4003408A0
:100B3000F7000130770283120319A62DF708031975
:100B4000AD2D023077020319F12DF82D8316B70170
:100B50008430B6008312EB24F92D8316B70181305F
:100B6000B6008312EB248316B7018230B6008312DD
:100B7000EB2401308316B7008030B6008312EB24DB
:100B800002308316B7008030B6008312EB240430A5
:100B90008316B7008030B6008312EB24083083162A
:100BA000B7008030B6008312EB2410308316B700F4
:100BB0008030B6008312EB2420308316B7008030DB
:100BC000B6008312EB2440308316B7008030B600A5
:100BD0008312EB2480308316B700B6008312EB2417
:100BE000F92D0F308316B7008730B6008312EB243F
:100BF000F92D8316032E83163208B4008312362D86
:100C00008316032E831683128A110A121A2E0A10D3
:100C10008A140A1582075B2D942DFB2D20302802A3
:100C2000FF3E03181B2E013E202E83163108B20012
:100C30008312532D1B2E871107128A110A122A2E96
:100C40000A108A140A158207152E2A088316B10085
:100C500083120E2E0730A9000130EF006B208A119D
:100C60000A16BD288316D608031D3A2E55082F3CB8
:100C700003184D2ED608031D4D2E5508303C031C7D
:100C80004D2E031D4A2ED408031D4D2E53080D3C36
:100C9000031C4D2ED801D701502E1030D800D7019B
:100CA000DE01831217248E308316E200A630E100A5
:100CB00083122E248316DE0183121724EF3083164D
:100CC000E200E10183122E248316DE018312172431
:100CD000F8308316E200E10183122E248316DE0130
:100CE0008312172483165708A638D90058088C3861
:100CF000DA00E2005908E10083122E248316560818
:100D0000DC005508DB005408DA005308D9008312D0
:100D1000482400348316DE0183121724843083169E
:100D2000E200A630E10083122E248316DE01831236
:100D3000172488308316E200A630E10083122E24A7
:100D40008316DE01831217240E308316E20055301D
:100D5000E10083122E248316DE01831217246E30E5
:100D60008316E200A730E10083122E248316DE01F1
:100D7000831217240E308316E200AA30E10083129A
:100D80002E248316DE01831217246E308316E200B0
:100D9000A730E10083122E248316DE01831217246C
:100DA00082308316E200A630E10083122E248316DF
:100DB000DE01831217248316E201E10183122E243F
:100DC0008316DE0183121724831623082507D30018
:100DD000D4008312C820831624082607D300D40029
:100DE0008312A7248316E201E10183122E248316C5
:100DF000DE018312172494308316E200A630E1004E
:100E000083122E2400348316CD08031D0B2F4C08AB
:100E10001F3C0318352FCD08031D342F4C082F3CE1
:100E2000031C342F7418342FDC013C30DB00DA0152
:100E30000630D900831248240C308316DE0083125A
:100E400017248316E201E10183122E2483164D0834
:100E5000D6004C08D5004B08D4004A08D3008312B2
:100E600032268A2674148316BA2F0030CA05F03051
:100E7000CB051F30CC050030CD05FA014D0CF90033
:100E80004C0CF8004B0CF700F90CF80CF70CF90CB3
:100E9000F80CF70CF90CF80CF70C7708CE004E0C98
:100EA000CF00CF0CCF0C1F30CF054E080739F8000C
:100EB0000130CE00F8080319612F0310CE0DF80B96
:100EC0005D2F8317A03083164F07840000084E055E
:100ED000003A031DB82FA0304F07840000084E04CD
:100EE0008000831283138316D101D001D108031D22
:100EF000B82F50083F3C031CB82F6400D2015208A1
:100F00003F3C031CB42F6400DC013C30DB00DA0101
:100F10000630D900831248240C308316DE00831279
:100F200017248316E201E10183122E2483164D0853
:100F3000D6004C08D5004B08D4004A08D3008312D1
:100F400032268A2683162908CA0700300318013082
:100F5000CB07003003180130CC07003003180130F4
:100F6000CD072908D2077F2FD00A0319D10A762F7F
:100F700083138316831200348316D1015108023C77
:100F8000031CD12F0310D00C0318CA2F8312071291
:100F9000CC2F831683120716871587118316D10A63
:100FA000BE2F0310D00C0318D92F83120712DB2F8A
:100FB000831683120716871583162108D40083121F
:100FC000C82083162208D4008312A7248711831611
:100FD0002308D4008312C82083162408D400831267
:100FE000A724003400308C1A0130F800003429089E
:100FF0000C1EF82F99002908EE060034EE06003486
:1010000083160716D10151080F3C031C15288312C3
:1010100087158711071A0E2803100F28031483164B
:1010200050088400800CD10A03280712831287110C
:10103000003483164C08013C03187728CD01023098
:101040004C024D02031841280D30DE008A11831234
:1010500017248A1583164B08CB0ACB0A8400840A0E
:101060000008CF0084030008CE004F08E2004E08BD
:10107000E1008A1183122E248A1502308316CD07CF
:101080001F280F30DE008A11831217248A15831659
:101090004B08CB0ACB0A8400840A0008CF008403E3
:1010A0000008CE004F08E2004E08E1008A118312CA
:1010B0002E248A158316D0018A118312BC278A1523
:1010C0008316E201E1018A1183122E248A150D3064
:1010D0008316DE008A11831217248A15FF308316C7
:1010E000E200E1008A1183122E248A1583168312EE
:1010F000003420302802FF3E0318132B013E182B2A
:1011000083163908BF003808BE003708BD0036080E
:10111000BC003A08C0003B08C100AD08031DD4283C
:101120003F08CD003E08CC003D08CB003C08CA007B
:101130008A11831203278A15831641083C07C200CF
:101140003D08C300003003180130C3073E08C40047
:10115000003003180130C4073F08C50000300318F1
:101160000130C50701304202C6004308C700003005
:10117000031C0130C7024408C8000030031C0130C2
:10118000C8024508C9000030031C0130C9024908E3
:10119000CD004808CC004708CB004608CA008A1199
:1011A000831203278A158316DC013C30DB00DA0149
:1011B0000630D9008A11831248248A150C30831610
:1011C000DE008A11831217248A158316E201E101D9
:1011D0008A1183122E248A1583163F08D6003E08F2
:1011E000D5003D08D4003C08D3008A118312322672
:1011F0008A158316BF08031D01293E082F3C0318DA
:101200000C2ABF08031D0C2A3E08303C031C0C2A84
:10121000031D1129BD08031D0C2A3C080D3C031CAD
:101220000C2A2D08F700F708831203192029013032
:1012300077020319202902307702031978290A2A34
:1012400083164008C2004108C3004208C500C4011B
:1012500043084402031876290F30DE008A118312F6
:1012600017248A15831645088400840A0008C700DD
:1012700084030008C6004708E2004608E1008A111E
:1012800083122E248A158316D0018A118312BC275B
:101290008A158316E201E1018A1183122E248A1530
:1012A0008316D0018A118312BC278A152A3083162F
:1012B000E200F630E1008A1183122E248A1583168B
:1012C000DE018A11831217248A158316E201E101D7
:1012D0008A1183122E248A15831644080139F700D7
:1012E0000310F70D7708C507C40A28290B2A0B2A13
:1012F00083164008C2004108C3004208C40003101E
:10130000C30CC3080319082A4408C40AC40A840089
:10131000840A0008FA0084030008C5007A08C600A1
:101320002B08C8000D30DE008A11831217248A159D
:1013300083164608E2004508E1008A1183122E2434
:101340008A158316D0018A118312BC278A15831649
:10135000E201E1018A1183122E248A150C308316D2
:10136000DE008A11831217248A1583164608E200CC
:101370004508E1008A1183122E248A158316D001B4
:101380008A118312BC278A158316E201E1018A11B2
:1013900083122E248A158316C80BCF29D1298312D4
:1013A000AE290E30DE008A11831217248A158316A7
:1013B0004608E2004508E1008A1183122E248A15AE
:1013C0008316D0018A118312BC278A158316E20185
:1013D000E1018A1183122E248A1509308316DE005A
:1013E0008A11831217248A15C7308316D0008312FE
:1013F000002009308316DE008A11831217248A1513
:10140000C7308316D000831200208316C3038129BE
:101410000B2A83128316112B2D08F700F70883126D
:1014200003191B2A0130770203191B2A02307702A5
:101430000319612A102B83163F08C5003E08C4001B
:101440003D08C3003C08C2004008C6004108C70070
:1014500042082805C900C9080319412A490827027A
:10146000CA0047020318362A4708CA004608CB00BC
:101470004A08CC008312192083164A08C7024A087A
:10148000C60747082805C8002808FF3AC705C70847
:101490000319562A4608CB002708CC0083121920CE
:1014A00083162708C6072708C702472AC808031952
:1014B000602A4608CB004808CC0083121920831606
:1014C000112B83163F08C5003E08C4003D08C30029
:1014D0003C08C2004008C6004108C7004608C800D2
:1014E0000310C70CC70803190E2B4808C80AC80AFE
:1014F0008400840A0008FA0084030008C9007A08FE
:10150000CA002A08CF000D30DE008A11831217248A
:101510008A1583164A08E2004908E1008A118312FD
:101520002E248A158316D0018A118312BC278A15AE
:101530008316E201E1018A1183122E248A150A30F2
:101540008316DE008A11831217248A15CD30831684
:10155000D0008312002008308316DE008A11831227
:1015600017248A15CE308316D000831200208316EC
:101570004D08CC004E08CB00CF030319C72A4908F9
:101580004B02031D832A4A084C02031D832A4F087D
:101590002A02D0002C08D1005008D2008A118312F0
:1015A00020218A1578088316CF000C30DE008A11BE
:1015B000831217248A1583164A08E2004908E100BD
:1015C0008A1183122E248A158316D0018A11831260
:1015D000BC278A158316E201E1018A1183122E24A9
:1015E0008A158316CF0BD52A0930DE008A118312A3
:1015F00017248A15CD308316D000831200200930BD
:101600008316DE008A11831217248A15CD308316C3
:10161000D000831200208316C703722A112B831275
:1016200083168312132B871107128A150A123E2B79
:101630000A148A140A11820780288316B4018312BF
:101640002C088316B30083122B088316B200831272
:101650002A088316B100043083126F028316B50086
:101660003408B9003308B8003208B7003108B600B2
:101670002D30BA003508BB00831279280730A90045
:101680000130EF008A116B208A158A110A16C628CC
:1016900020302802FF3E0318802B013E852B831645
:1016A0003808BE003708BD003608BC003508BB004E
:1016B0003908BF003A08C0003E08D6003D08D500F2
:1016C0003C08D4003B08D3008A11831232268A15C5
:1016D0008316C1014008410203187E2B0930DE0049
:1016E0008A11831217248A1583163F084107C20006
:1016F000D000831200208316C10A6A2B8312802B2C
:10170000871107128A150A12AC2B0A148A140A11BF
:1017100082074F2B8316B40183122C088316B30063
:1017200083122B088316B20083122A088316B10095
:1017300083122D08EF0083163408B8003308B70071
:101740003208B6003108B5002D30B90083126F0899
:101750008316BA008312482BC430A9000430EF0767
:101760008A116B208A158A110A16D0288316DE0189
:101770008A11831217248A1583164308C4000E3079
:10178000C500E2004308E1008A1183122E248A1565
:101790008316DE018A11831217248A156E30831690
:1017A000E200A830E1008A1183122E248A158316E4
:1017B000DE018A11831217248A1584308316E20011
:1017C000A630E1008A1183122E248A158316DE01C9
:1017D0008A11831217248A150E308316E2005530C1
:1017E000E1008A1183122E248A158316DE018A11E4
:1017F000831217248A156E308316E200A730E100A9
:101800008A1183122E248A158316DE018A1183120F
:1018100017248A150E308316E200AA30E1008A11DF
:1018200083122E248A158316DE018A11831217244F
:101830008A156E308316E200A730E1008A11831208
:101840002E248A158316DE018A11831217248A1525
:1018500082308316E200A630E1008A1183122E2422
:101860008A15003420302802FF3E0318F42D013E73
:10187000F92D83163508B9003408B8003608BA00C7
:101880003708BB0000302E180130F700F70883122C
:1018900003194F2C013077020319F22CF12D831616
:1018A0003908BD003808BC003A08BE003B08BF003C
:1018B000DE018A11831217248A159E308316E200F6
:1018C000A630E1008A1183122E248A158316DE01C8
:1018D0008A11831217248A159C308316E200A630E1
:1018E000E1008A1183122E248A158316C0013F0855
:1018F00040020318F12CDE018A11831217248A1585
:1019000083163D08FA003C08BC0A0319BD0AC10051
:101910007A08C2004108F70042080039FA0041087D
:10192000C3007A080E38C400E2004108E1008A11C1
:1019300083122E248A158316DE018A11831217243E
:101940008A156E308316E200A930E1008A118312F5
:101950002E248A1583163E08400784000008C10023
:10196000C3008312B6238316DE018A118312172463
:101970008A158316E201E1018A1183122E248A1549
:101980008316DE018A11831217248A158316230811
:101990002507C100D4008A118312C8208A15831636
:1019A00024082607C100D4008A118312A7248A15AF
:1019B0008316E201E1018A1183122E248A1583160F
:1019C000DE018A11831217248A1594308316E200EF
:1019D000A630E1008A1183122E248A158316C00ACC
:1019E000772CF22D83163908BD003808BC003A0860
:1019F000BE003B08BF00DE018A11831217248A153E
:101A00009E308316E200A630E1008A1183122E2454
:101A10008A158316DE018A11831217248A159C30D9
:101A20008316E200A630E1008A1183122E248A1563
:101A30008316C0013F0840020318EF2D0230C10099
:101A4000DE018A11831217248A1583163C08F700D9
:101A50003D080039FA003C08C2007A080E38C3007D
:101A6000E2003C08E1008A1183122E248A158316B5
:101A7000DE018A11831217248A156E308316E20064
:101A8000A930E1008A1183122E248A158316DE0103
:101A90008A11831217248A1583163D08C200C301D8
:101AA0003D08F70043080039FA003D08C4007A08F1
:101AB0000E38C500E2003D08E1008A1183122E2491
:101AC0008A158316BC0A0319BD0ADE018A11831226
:101AD00017248A156E308316E200AA30E1008A11BD
:101AE00083122E248A150F30F700F70B752D8316FD
:101AF0003E08400784000008C200C3008312B623DA
:101B0000831641080239003A0319CA2DDE018A11F1
:101B1000831217248A1550308316E200A630E100A4
:101B20008A1183122E248A150230F700F70B962DA6
:101B3000000000008316DE018A11831217248A1523
:101B40006E308316E200F530E1008A1183122E24F4
:101B50008A158316DE018A11831217248A158316CB
:101B6000E201E1018A1183122E248A1502308316C4
:101B7000DE008A11831217248A15C1308316D00023
:101B8000831200200230F700F70BC42D0000000084
:101B9000802D83162308D4008A118312C8208A1549
:101BA00083162408D4008A118312A7248A15831669
:101BB000DE018A11831217248A1594308316E200FD
:101BC000A630E1008A1183122E248A150230F70014
:101BD000F70BE82D000000008316C00A1A2DF22D25
:101BE000831283168312F42D871107128A150A12A5
:101BF000142E0A148A100A158207392C2B08831612
:101C0000B20083122A088316B100033083126F02D8
:101C10008316B3003208B5003108B4002C30B6008A
:101C20003308B7008312322C0730A9000130EF00CF
:101C30008A116B208A158A110A16DA288316DE01AA
:101C40008A11831217248A1580308316E200A63089
:101C5000E1008A1183122E248A158316DE018A116F
:101C6000831217248A1550308316E200A830E10051
:101C70008A1183122E248A158316DE018A1183129B
:101C800017248A156E308316E200F530E1008A11C0
:101C900083122E248A158316DE018A1183121724DB
:101CA0008A158316E201E1018A1183122E248A1516
:101CB00002308316DE008A11831217248A158316D8
:101CC0004108D00083120020003420302802FF3E5B
:101CD0000318762F013E7B2F83163408B800330893
:101CE000B7003508B9003608BA0000302E180130A8
:101CF000F700F70883120319822E013077020319C7
:101D0000E82E732F83163808BC003708BB0039084B
:101D1000BD003A08BE00DE018A11831217248A151D
:101D20009E308316E200A630E1008A1183122E2431
:101D30008A158316DE018A11831217248A159C30B6
:101D40008316E200A630E1008A1183122E248A1540
:101D50008316BF013E083F020318E72EDE018A11F9
:101D6000831217248A1583163C08FA003B08BB0A25
:101D70000319BC0AC0007A08C1004008F7004108F6
:101D80000039FA004008C2007A080E38C300E200A9
:101D90004008E1008A1183122E248A158316DE0181
:101DA0008A11831217248A156E308316E200A93037
:101DB000E1008A1183122E248A1583163D08BD0A7C
:101DC000C000C10083121E268316BF0AAA2E742FDC
:101DD00083163808BC003708BB003908BD003A0834
:101DE000BE00DE018A11831217248A159E308316E5
:101DF000E200A630E1008A1183122E248A15831690
:101E0000DE018A11831217248A159C308316E200A2
:101E1000A630E1008A1183122E248A158316BF0191
:101E20003E083F020318712FDE018A118312172426
:101E30008A1583163B08F7003C080039FA003B0876
:101E4000C0007A080E38C100E2003B08E1008A11A8
:101E500083122E248A158316DE018A118312172419
:101E60008A156E308316E200A930E1008A118312D0
:101E70002E248A158316DE018A11831217248A15EF
:101E800083163C08C000C1013C08F7004108003936
:101E9000FA003C08C2007A080E38C300E2003C0891
:101EA000E1008A1183122E248A158316BB0A0319B6
:101EB000BC0ADE018A11831217248A156E3083163C
:101EC000E200AA30E1008A1183122E248A158316BB
:101ED0003D08BD0AC000C10083121E268316BF0A3A
:101EE000102F742F831283168312762F87110712F7
:101EF0008A150A12972F0A148A140A1582076C2E63
:101F00002B088316B20083122A088316B1008312AD
:101F10002C08EF0083163208B4003108B3002C30CF
:101F2000B50083126F088316B6008312652EE23067
:101F3000A9000330EF078A116B208A158A110A164F
:101F4000E4288A114B208A15D030A900AA01AB01E0
:101F5000AC01AD010530EF008A116B208A158A11A2
:101F60000A16EE288A1174228A15D030A900013091
:101F7000AA00AB01AC01AD010530EF008A116B2066
:101F80008A158A110A16F82883165F1464008312D2
:101F9000071EDE2F640083165E08DE03003A031D71
:101FA000D62F5F108312DE2FDD2F83164D30F70002
:101FB000F70BD82F000000008312C82F00308316C3
:101FC0005F180130F8008312003408300C1EE62F31
:101FD00099008316480883120C1EEC2F99000034D8
:101FE00003300C1EF12F99008316380883120C1E43
:101FF000F72F9900831638088312EE00003400345E
:1020000001308316B000B4012930B500B408031DB7
:1020100056280A12831254200A1678088316B10033
:102020003108043C03191C280A12831254200A1692
:1020300078088316B10010280A12831254200A1659
:102040007808EF008316B300B20183126F0883167D
:10205000320203183D283508B6000A1283125420B4
:102060000A16831636088400780880003508840034
:102070000008B306B50AB20A25280A1283125420B2
:102080000A1678088316B306031D4F280130B400E2
:10209000063083120C1E4A289900542883160530F6
:1020A00083120C1E512899008316062883122908D2
:1020B000103C031D5F280A12B4200A16FE282908C6
:1020C000113C031D67280A12DD280A16FE2829087C
:1020D000123C031D6F280A1247290A16FE282908F8
:1020E000143C031D77280A12D8290A16FE2829084D
:1020F000153C031D7F280A12A4210A16FE28290870
:10210000173C031D87280A12F2290A16FE282908FF
:10211000183C031D8F280A12342A0A16FE282908A3
:102120001A3C031D97280A12612A0A16FE2829085C
:102130001B3C031D9F280A126A2A0A16FE2829083A
:10214000413C031DA7280A12B12B0A16FE282908B4
:10215000403C031DAF280A12C52B0A16FE28290889
:10216000473C031DB7280A120B2C0A16FE28290823
:10217000433C031DBF280A12252E0A16FE282908F3
:10218000423C031DC9280A128A151D2B0A168A1102
:10219000FE282908443C031DD3280A128A158A2BDD
:1021A0000A168A11FE282908453C031DDD280A125B
:1021B0008A15FE2D0A168A11FE282908463C031DA1
:1021C000E7280A128A15802F0A168A11FE28290884
:1021D000503C031DF1280A128A15A12F0A168A11F4
:1021E000FE282908513C031DFB280A128A15B22F2C
:1021F0000A168A11FE288316B0018312831630084E
:10220000F80083128A150A16152F8316560DD7006B
:10221000D70DD70DF830D7050716FF30DE000A12AC
:102220008A158312C4270A168A118316D901D80188
:1022300059087102031C2A29031D2229580870021B
:10224000031C2A290230F700F70B2429D80A0319A6
:10225000D90A1829831287158316D901D80159087C
:102260007102031C4229031D392958087002031CFE
:1022700042290630F700F70B3B290000D80A031962
:10228000D90A2F298312071A472903104829031452
:102290008316DA0DDB0DDC0D07128312071283168D
:1022A000560B58290310D20D031C582907166D2907
:1022B0005608023C031D63290310D20DD30D031CE5
:1022C000632907166D295608033C031D6D29031069
:1022D000D20DD30DD40D0318071683128711831660
:1022E000D901D80159087102031C8529031D7C29D5
:1022F00058087002031C85290630F700F70B7E2969
:102300000000D80A0319D90A72290716D70B2A29FF
:1023100007165A08F7005B08F8005C08F9005D082A
:10232000FA00831200348316BB01BC01F101733043
:10233000F000FF30DE000A128A158312C4270A1645
:102340008A11F8080319052A8316D501D401103023
:10235000D300D2010230D60083120521831607165E
:102360008312071AB1298316BC01BB01831287159A
:10237000F3010130F200071AC629F20A0319F30A21
:10238000720873040319C6296400BB29071AD129EE
:10239000F20A0319F30A720873040319D1296400BD
:1023A000C6298312071EE3298316BB0A0319BC0A38
:1023B0003B083C040319E32912306400FF3E031D6F
:1023C000DD290000D12983128711720873040319D3
:1023D000002A83163B083C04031DF0298312002ABF
:1023E0003C0CF1003B0CF000F10CF00CF10CF00C8B
:1023F000F10CF00CF10CF00C0730F105042A8312FB
:10240000F1017330F0008316831283163B08F80045
:102410003C08F90083120034831605118312051558
:1024200083168512831285168316861083128614EE
:10243000F1017330F00020302802FF3E0318602ABB
:10244000013E812A0A124B200A1687150A127422AD
:102450000A160230F700F70B2B2A00000000871144
:10246000FF308316DE000A128A158312C4270A166B
:102470008A110A124B200A1687150A1274220A16AC
:102480000230F700F70B422A000000008711831684
:10249000D501A030D400D301D2010330D60083127D
:1024A00005211F30F9050030FA057A088316BA00B5
:1024B0007908B9007808B8007708B7008312602A55
:1024C0009321FF308316DE000A128A158312C42777
:1024D0000A168A11F808031D742A8316BA01FF3000
:1024E000B900B800B700831283163708F700380820
:1024F000F8003908F9003A08FA0083128A110A161E
:102500008B2A0A108A140A118207222AB2308316F3
:10251000B60083120C2A7A088316B5007908B40035
:102520007808B3007708B200D0308312A900831670
:10253000DE010A128A158312C4270A168A11F808C6
:102540000319A42A0030A52A0130AA0083163608F0
:10255000B60A840000088312AB0083163608B60A58
:10256000840000088312AC0083163608840000083B
:102570008312AD000530EF000A126B200A168A158F
:102580000A16472E8316BA01FF30B900B800B7000B
:10259000DE010A128A158312C4270A168A11F80866
:1025A000031D022B87151E30F700F70BD52A0000FC
:1025B000871120302802FF3E0318F92A013E0F2B15
:1025C0008316D501A030D400D301D2010330D60048
:1025D000831205211F30F9050030FA057A088316A9
:1025E000BA007908B9007808B8007708B7008312F4
:1025F000F92AFF308316DE000A128A158312C427D7
:102600000A168A1183163708F7003808F8003908C7
:10261000F9003A08FA0083128A110A16192B0A14D3
:102620008A140A118207E02AB2308316B600831298
:10263000C22A7A088316B5007908B4007808B30076
:102640007708B200D0308312A9008316DE010A1287
:102650008A158312C4270A168A11F8080319322B27
:102660000030332B0130AA0083163608B60A8400E6
:1026700000088312AB0083163608B60A84000008EF
:102680008312AC0083163608840000088312AD0064
:102690000530EF000A126B200A168A150A164F2E13
:1026A0000830F7000718522B8316CC01F717682B58
:1026B000F713682B03108312071803148316CC0C2E
:1026C0007717682B7713F70B5A2B4C08F800752BEC
:1026D0007930F71B2130F800F80B6C2B000000005C
:1026E000F71B582B771B622B5A2B83128A150A165D
:1026F000A62807100830F800000000000000F817B6
:10270000922BF8138316C90C831203180714031CA9
:1027100007107817922B7813F80B822B000000001B
:102720000000071479308400840B942B0000000013
:10273000F81B812B781B8B2B8A150A164229FF3038
:102740008316C600C700C800C901DE010A128A1537
:102750008312C4270A168A11F8080319CF2B2030D8
:102760002802FF3E0318CF2B013EDA2B8316D5013A
:10277000A030D400D301D2010330D600831205214A
:102780001F30F9050030FA057A088316C900790868
:10279000C8007808C7007708C6008312CF2B8316BD
:1027A0004608F7004708F8004808F9004908FA0009
:1027B000831200340A148A140A118207B62B831676
:1027C0003714B230B60083126F08053C031DF42B9A
:1027D0002D080139003A031DF12B83163710F32B16
:1027E00083128316371483128316BB0183122C08BD
:1027F0008316BA0083122B088316B90083122A08A5
:102800008316B800003037180130BC003B08C00008
:102810003A08BF003908BE003808BD003C08C100B6
:102820008A15831200288A117A088316B500790860
:10283000B4007808B3007708B200D0308312A90042
:102840008316DE010A128A158312C4270A168A111A
:10285000F80803192D2C00302E2C0130AA00831605
:102860003608B60A840000088312AB0083163608C7
:10287000B60A840000088312AC0083163608840070
:1028800000088312AD000530EF000A126B200A1613
:102890008A150A16572EFF308316DE000A128A1593
:1028A0008312C4270A168A11F8080319862C2030CF
:1028B0002802FF3E0318862C013EA62C8316D50164
:1028C000C030D400D301D2010330D60083120521D9
:1028D0001E30F700F70B6A2C00008316D501A030DC
:1028E000D400D301D2010330D600831205211F305A
:1028F000F9050030FA057A088316BA007908B9009C
:102900007808B8007708B7008312862CFF3083164A
:10291000DE000A128A158312C4270A168A11F808E3
:10292000031D992C8316BA01FF30B900B800B70017
:10293000831283163708F7003808F8003908F900C1
:102940003A08FA0083128A110A16B02C0A108A106B
:102950000A1582075E2CB2308316B60083124B2C08
:102960007A088316B5007908B4007808B3007708B0
:10297000B200D0308312A9008316DE010A128A1534
:102980008312C4270A168A11F8080319C92C0030CB
:10299000CA2C0130AA0083163608B60A8400000843
:1029A0008312AB0083163608B60A8400000883122F
:1029B000AC0083163608840000088312AD00053091
:1029C000EF000A126B200A168A150A165F2E6E088F
:1029D0000C1EE82C99000A1254200A167808063CAE
:1029E000031DEB2C0034831283162908F800831290
:1029F000003465200A168A150A166D28FF3FFF3F2E
:102A000084011F308305073083169F000230990030
:102A100022309800903083129800A001A10110305C
:102A2000A2003030A3008A30A400A501A6012D30F9
:102A3000A700FF30EF00EF106F08831687008312A6
:102A40008714023083169900223098009030831248
:102A5000980002308316990022309800903083123B
:102A600098000F30F70007308101813084000008A2
:102A7000F0390738800064000008F03977048000DE
:102A8000A32564009626412D63000C1E452D990058
:102A90007A2D0530F6007608063C03197A2D8C1A3B
:102AA000532D64004F2D8C1E532D1A088316A00041
:102AB0008312981C612D1A088316A0008312181225
:102AC000181683162008F800831200342808073CE3
:102AD000031D6F2D07300C1E6B2D9900A22D0530A4
:102AE000FC007C08063C0319A22D7C08053C031D54
:102AF0009E2D2830FE006E08F60004300C1E7E2D40
:102B000099006E080C1E822D9900FD016E087D0251
:102B100003189A2D7E08840000088316A0008312F3
:102B20000C1E902D99007E0884000008F606FE0A0F
:102B3000FD0A862D76080C1E9B2D99004F257808DE
:102B4000FC00712D0034B130A8000130EE00662584
:102B50000034F3012830F400F308031DE42D4F2561
:102B60007808F0007008043C0319BA2D4F25780846
:102B7000F000B22D4F257808EE006E08F200F1014A
:102B80006E0871020318D22D7408F5004F257508E0
:102B9000840078088000740884000008F206F40AB3
:102BA000F10AC02D4F257808F206F208031DDF2D2B
:102BB0000130F30006300C1EDB2D9900E32D0530AB
:102BC0000C1EE02D9900AC2D003403306E02003A4B
:102BD0000319502EF1012A08F0007008F1002908AD
:102BE000F0002B30F5000330F4006E087402031877
:102BF000502E7508F50A84000008FA01F2007A08E0
:102C0000F3007508F50A84000008F600F300710867
:102C1000143C03180F2E7108163C03184A2E710835
:102C20001F3C031C4A2EF108031D292E7008033C8B
:102C3000031C292E0310700DF900710DFA0079089C
:102C4000203E8400840A7308800084037208800098
:102C50004A2E700803178D0071088F0072088C00CF
:102C600073088E0083168C170C15831203130B0840
:102C7000F8008B138316031755308D00AA308D0092
:102C80008C14000000008C18432E0C11780883125D
:102C900003138B04F00A0319F10A0230F407F52D2F
:102CA0000730A8000130EE0066250034F0017008FE
:102CB000033C031C8C2EF2017008F1000310700D10
:102CC000F700203E8400840A0008F4008403000812
:102CD000F300700803178D0072088F0073088C00D2
:102CE00074088E0083168C170C15831203130B08BF
:102CF000F8008B138316031755308D00AA308D0012
:102D00008C14000000008C18832E0C11780883129C
:102D100003138B04F00A572E8C2E00342808A900C8
:102D2000FF30A8000230EE0066250034A9252808EF
:102D3000F700313077020319A62E323077020319DB
:102D4000A82E333077020319AA2EAC2EA325AE2E5F
:102D5000E525AE2E5626AE2E8E26AE2E0034FF3F33
:102D6000FF3FFF3FFF3FFF3FFF3FFF3FFF3FFF3F73
:102D7000FF3FFF3FFF3FFF3FFF3FFF3FFF3FFF3F63
:102D8000FF3FFF3FFF3FFF3FFF3FFF3FFF3FFF3F53
:102D9000FF3FFF3FFF3FFF3FFF3FFF3FFF3FFF3F43
:102DA000FF3FFF3FFF3FFF3FFF3FFF3FFF3FFF3F33
:102DB000FF3FFF3FFF3FFF3FFF3FFF3FFF3FFF3F23
:102DC000FF3FFF3FFF3FFF3FFF3FFF3FFF3FFF3F13
:102DD000FF3FFF3FFF3FFF3FFF3FFF3FFF3FFF3F03
:102DE000FF3FFF3FFF3FFF3FFF3FFF3FFF3FFF3FF3
:102DF000FF3FFF3FFF3FFF3FFF3FFF3FFF3FFF3FE3
:102E0000B2308316B60083129F237A088316B5006A
:102E10007908B4007808B3007708B200D030831284
:102E2000A9008316DE010A128A158312C4270A1626
:102E30008A11F80803191E2F00301F2F0130AA0035
:102E400083163608B60A840000088312AB00831686
:102E50003608B60A840000088312AC0083163608D0
:102E6000840000088312AD000530EF000A126B20C9
:102E70000A168A150A16672E8316C201FF30DE0075
:102E80000A128A158312C4270A168A11F808031930
:102E9000562F8316D501D401D301D2010130D600BB
:102EA0008312052177088316C20083128316420815
:102EB000F80083120034FF308316DE000A128A15F0
:102EC0008312C4270A168A11F8080319852F83165E
:102ED0003F08F70040080F39FA003F08C2007A089F
:102EE0004038C300C401C5014508D5004408D400DA
:102EF0004308D3003F08D2000230D60083120521D8
:102F00003C2778088316C1008312FF308316DE0049
:102F10000A128A158312C4270A168A11F808031D9B
:102F2000952FFF308316C100831283164108F800E5
:102F30008312003429308316B40083122B088316C1
:102F4000B30083122A088316B20083122C0883165A
:102F5000B60003303607B700B8000A128A1583128C
:102F6000F0270A168A11831634088400E0308000A6
:102F70000A128312F7270A16831634088400831274
:102F80002A0880000A12F7270A16831634088400DC
:102F900083122B0880000A12F7270A1683163408BA
:102FA000B7003308C0003208BF0083125B278316C6
:102FB00037088400780880000A128312F7270A165F
:102FC00001308316B500360835020318F72F340890
:102FD000B70083123C2783163708840078088000E6
:102FE0000A128312F7270A168316B50AE32F8312F3
:102FF000E7248A150A166F2EFF3FFF3FFF3FFF3F72
:10300000FF308316C200C300C400C501DE010A12EE
:103010008312C4270A16F8080319772820302802DB
:10302000FF3E03187728013E822983164008C90015
:103030003F08C8003E08C7003D08C600FF30CA0070
:10304000CB00CC00CD014608F7004708F80048083F
:103050001F39F90049080039FA004608CE00470830
:10306000CF0079088038D0007A08D100D500500808
:10307000D4004708D3004608D2000330D6008A1196
:10308000831205218A158316DE010A128312C427D2
:103090000A16F808031964288316D501A030D40055
:1030A000D301D2010330D6008A11831205218A157B
:1030B00077088316CA007808CB0079081F39CC003E
:1030C0007A080039CD00831283164A08F7004B08AE
:1030D000F8004C08F9004D08FA007A08C500790894
:1030E000C4007808C3007708C200831277288316CB
:1030F000C10803195629461046185629DE010A123E
:103100008312C4270A16F80803198828831656293B
:10311000C7308316C8004914C9108610831286145C
:1031200083160714F41C9928480884000130800095
:10313000D428C918D428640083120718AF2883162E
:1031400048088400CB008A118312502B8A158316FD
:103150004B08840078088000C914D32883120A120F
:103160008A11F2270A168A15F8080319C5280A12C7
:103170008A1154200A168A157808023C031DC428B7
:103180008316C91449108312D2288316DE010A124D
:103190008312C4270A16F8080319D2288316C91403
:1031A0004910831283169928003049180130F8001D
:1031B000F808031952294708F700013077028312F3
:1031C0000319E328492901308316C8000A12831223
:1031D000E5270A16C7308316C8004914C910C91854
:1031E0003129DE010A128312C4270A16F8080319CE
:1031F000FB28831631290A128A11F2270A168A152A
:10320000F80803192F2983164808CA000A128A11E0
:10321000831254200A168A1583164A0884007808F7
:103220008000480884000008083C031D262948083F
:10323000CA000A128A11831254200A168A158316AC
:103240004A08840078088000C9142E2948088400A0
:103250000008023C031D2E29C9144910831283164D
:10326000EF28003049180130F800F8080319452903
:10327000F4104708C800861407104808C9008A11CE
:103280008312792B8A1548298316F4144614831265
:10329000502983164708C8000A128312E5270A1628
:1032A000542983164614831283167C28420F5F2903
:1032B000430F5F29440F5F29C50803196929420F8D
:1032C0007629430F7629C408031D7629C508031DF6
:1032D00076298A1183129F238A157A088316C500DE
:1032E0007908C4007808C3007708C2004208F700D4
:1032F0004308F8004408F9004508FA0083128A11CF
:103300000A16132C0A148A100A1182071528FF3096
:103310008316DE000A128312C4270A16F80803195E
:10332000C82983164108F70042080F39FA004108FE
:10333000C4007A085038C500C601C7014708D50047
:103340004608D4004508D3004408D2000230D60015
:103350008A11831205218A15FF308316DE000A12B6
:103360008312C4270A1683164308C4006030C500C0
:10337000C601C7014708D5004608D4004508D30058
:103380004408D2000230D6008A11831205218A1522
:1033900000342B088316B40083122A088316B30066
:1033A0000330B20083126F08831632020318F1292A
:1033B0003408FA003308B30A0319B40AB5007A08CE
:1033C000B6002930320784000008B7003608C20072
:1033D0003508C1003708C300831287218316B20A5B
:1033E000D22907308312A9000130EF000A128A1196
:1033F0006B200A168A158A150A16762E831640083F
:10340000F70041080339FA004008C2007A08203862
:10341000C300C401C5014508D5004408D4004308D1
:10342000D3004008D2000230D6008A118312052151
:103430008A158316D501D401D3010230D2000130A0
:10344000D6008A11831205218A157708F800003406
:103450008316BC01FF30DE000A128312C4270A164D
:10346000F8080319462A20302802FF3E0318462A8E
:10347000013E4D2A83163B08C1003A08C000831262
:10348000FE2178088316BC008312462A83163C0866
:10349000F80083128A150A16A02A0A108A140A1143
:1034A00082073A2A29308316B40083122B08831628
:1034B000B30083122A088316B20083122C088316E5
:1034C000B60003303607B700B8000A128312F0279F
:1034D0000A16831634088400E23080000A128A112A
:1034E0008312F7270A168A1583163408840083127C
:1034F0002A0880000A128A11F7270A168A158316ED
:103500003408840083122B0880000A128A11F727DE
:103510000A168A158316B501360835020318AE2A35
:103520003408B7003308FA003208B20A0319B30AA4
:10353000B8007A08B900BB003808BA008312282AFC
:10354000831637088400780880000A128A118312D3
:10355000F7270A168A158316B50A8C2A8A11831250
:10356000E7248A158A150A167C2EFF308316DE00A2
:103570000A128312C4270A16F80803190B2B2030ED
:103580002802FF3E03180B2B013E0E2B8316360834
:10359000BA003508B9003708BB003808BC00BD01C7
:1035A0003C083D020318092B3D083907BE003A08C4
:1035B000BF000318BF0A3F08C1003E08C0008312C5
:1035C000FE2183163B083D0784000008BE00BF00B3
:1035D000FF30DE000A128312C4270A16F808031906
:1035E000062B83163F08C0003030C100C201C30162
:1035F0004308D5004208D4004108D3003F08D20058
:103600000230D6008A11831205218A158316BD0A5D
:10361000D02A83120B2B8A150A16292B0A148A1416
:103620000A118207C62A2B088316B30083122A08C0
:103630008316B200033083126F028316B40033087E
:10364000B6003208B5002C30B7003408B800831239
:10365000B52A0730A9000130EF000A128A116B2049
:103660000A168A158A150A16822EFF308316DE0086
:103670000A128312C4270A16F8080319A52B203052
:103680002802FF3E0318A52B013EA82B83163A08FB
:10369000C0003908BF003808BE003708BD003B082D
:1036A000C1003C08C2000310BF0CBE0CBD0C3D089D
:1036B000F7003E08F8003F081F39F90040080039BC
:1036C000FA003D08C4003E08C5007908D038C6009D
:1036D0007A08C700D5004608D4003E08D3003D084C
:1036E000D2000330D6008A11831205218A15831671
:1036F000D501E030D400D301D2010330D6008A11C5
:10370000831205218A158316C30142084302031858
:10371000A32B4108C10AC10AC400D501E030D4007E
:10372000D301D2010330D6008A11831205218A15F4
:1037300083164408840077088000840A7808800093
:103740000230C307852B8312A52B8A150A16CF2BAF
:103750000A148A140A118207462B8316B6018312B3
:103760002C088316B50083122B088316B40083122D
:103770002A088316B30083122D08EF00831636083B
:10378000BA003508B9003408B8003308B7002D3046
:10379000BB0083126F088316BC008312352BC43024
:1037A000A9000430EF070A128A116B200A168A1545
:1037B0008A150A16882EFF308316DE000A1283123D
:1037C000C4270A16F8080319462C20302802FF3EA9
:1037D0000318462C013E492C83163B08C1003A08C9
:1037E000C0003908BF003808BE003C08C2003D08D0
:1037F000C3000310C00CBF0CBE0C3E08F7003F080E
:10380000F80040081F39F90041080039FA003E0865
:10381000C5003F08C6007908D038C7007A08C8003C
:10382000D5004708D4003F08D3003E08D20003303B
:10383000D6008A11831205218A158316C401430814
:1038400044020318442C4208C20AC20A8400840AB3
:103850000008FA0084030008C5007A08C600F030AA
:10386000C700C8014808D5004708D4004608D3005F
:103870004508D2000330D6008A11831205218A152B
:1038800002308316C4071F2C8312462C8A150A1691
:103890006F2C0A108A100A158207EC2B8316B601CA
:1038A00083122C088316B50083122B088316B400EC
:1038B00083122A088316B300043083126F02831622
:1038C000B7003608BB003508BA003408B900330821
:1038D000B8002D30BC003708BD008312DB2B073049
:1038E000A9000130EF000A128A116B200A168A150E
:1038F0008A150A168E2E2A308316B200973083124C
:10390000A90083163208B3008A11831293218A1505
:10391000831633088400840A7908800084037808B9
:10392000800003308312EF000A128A116B200A16FE
:103930008A158A150A16942EFF308316DE000A12A5
:103940008312C4270A16F80803190D2D2030280207
:10395000FF3E03180D2D013E102D83163508B900CA
:103960003708BA003808BB000F30C000FC30BF0079
:103970008A1183125B278A1578088316BC000F30E2
:10398000C200FC30C1003908C300831287218316AE
:10399000BD013B083D020318042D3A083D07BE0057
:1039A0000F30C000FD30BF008A1183125B278A15DB
:1039B00083163E0884007808800001303D073A07EE
:1039C000BF008A1183123C278A1583163F088400A2
:1039D0007808800002303D073A07BF008A11831241
:1039E0003C278A1583163F08840078088000B90AAE
:1039F0000F30C200FC30C1003908C3008312872198
:103A000003308316BD07C92C0F30C200FC30C10043
:103A10003C08C300831287210D2D8A150A16302D0C
:103A20000A148A100A158207AD2C2A308316B200B8
:103A300083122C08EF00831632088400840A0008E1
:103A4000B40084030008B3003408B6003308B5009E
:103A50002C30B70083126F088316B80083129C2C99
:103A6000E630A9000330EF070A128A116B200A160C
:103A70008A158A150A169A2EFF308316DE000A125E
:103A80008312C4270A16F8080319A82D203028022B
:103A9000FF3E0318A82D013EAB2D83163608BA0051
:103AA0003808BB003908BC000F30C000FC30BF0034
:103AB0008A1183125B278A1578088316BD00BE0120
:103AC0003C083E0203189F2D3A08BA0ABF000F3087
:103AD000C200FC30C1003F08C30083128721831657
:103AE0003B083E0784000008BF000F30C200FD30D5
:103AF000C1003F08C30083128721013083163E07AF
:103B00003B0784000008C0000F30C200FE30C10037
:103B10004008C30083128721023083163E073B070B
:103B200084000008C0000F30C200FF30C100400810
:103B3000C3008312872103308316BE07602D0F3028
:103B4000C200FC30C1003D08C30083128721A82DAC
:103B50008A150A16CA2D0A148A100A1582074D2DD5
:103B60002A308316B20032088400840A0008B400A8
:103B700084030008B300033083126F028316B5007C
:103B80003408B7003308B6002C30B8003508B90047
:103B900083123C2D0730A9000130EF000A128A1170
:103BA0006B200A168A158A150A16A02E8316B201F2
:103BB0003208033C031C282EB4013208B300031062
:103BC000320DF700B500350A0A128A11831235202A
:103BD0000A168A15FA00831635080A128A1183120A
:103BE00035200A168A158316B6007A08B7003308FE
:103BF000831203178D0083160313340883120317EF
:103C00008F00831603133608831203178C00831664
:103C100003133708831203178E0083168C170C15B5
:103C2000831203130B08F8008B1383160317553008
:103C30008D00AA308D008C14000000008C181E2E00
:103C40000C117808831203138B048316B20AD82D43
:103C50008A01831282018A150A16A62E2908AA0053
:103C6000FF30A9000230EF000A128A116B200A16F9
:103C70008A158A150A16A82E8316B108031DA92EC7
:103C800083122908523C031D492E8A11862A8A155F
:103C9000A82E2908533C031D512E8A11142B8A1576
:103CA000A82E2908543C031D592E8A11DF2B8A1592
:103CB000A82E2908553C031D612E8A11AB2C8A15AC
:103CC000A82E2908563C031D692E8A11002F8A153B
:103CD000A82E2908603C031D712E8A119A2F8A157F
:103CE000A82E2908613C031D772EC929A82E290872
:103CF000623C031D7D2E522AA82E2908633C031D19
:103D0000832E132BA82E2908653C031D892EAD2B6D
:103D1000A82E2908643C031D8F2E4E2CA82E29089E
:103D2000663C031D952E7B2CA82E2908673C031D9D
:103D30009B2E152DA82E2908683C031DA12EB02D01
:103D4000A82E2908313C031DA72ED62DA82E2E2ED5
:103D5000831683128A150A161C2F84011F308305CF
:103D6000073083169F00023099002230980090306F
:103D70008312980002308316990022309800903008
:103D800083129800023083169900223098009030F8
:103D900083129800023083169900223098009030E8
:103DA00083129800023083169900223098009030D8
:103DB000831298007330F000F101F4100714071417
:103DC000993083168700103086000B308500B5309F
:103DD000831290008F018E0183160C14C030831261
:103DE0008B040F30F7000730810181308400000818
:103DF000F0390738800064000008F039770480004B
:103E00000A128A114B200A168A150A128A11B42046
:103E10000A168A150B138B138B1B0B2F83160C1092
:103E20008312061564008A1100288A157808831603
:103E3000B000B10083123C2E122F63000319912FA2
:103E4000313077020319932F952F0A128A11AE2071
:103E50000A168A15962F0A128A11D7200A168A1571
:103E6000962F0A128A113F210A168A15962F0A12D6
:103E70008A11CC210A168A15962F0A128A119821C6
:103E80000A168A15962F0A128A11E4210A168A1533
:103E9000962F0A128A1124220A168A15962F0A12C0
:103EA0008A1184220A168A15962F0A128A119422E0
:103EB0000A168A15962F0A128A11C4220A168A1522
:103EC000962F0A122B220A16962F0A1222230A165E
:103ED000962F0A128B240A16962F0A120B260A1600
:103EE000962F8A113E208A15962F0A128A11F127E1
:103EF0000A168A15962F0A12C9270A16962F8A11B2
:103F000000278A15962F0020962F8E20962FD920D5
:103F1000962F7D21962F3A22962FBE22962F52233E
:103F2000962FE123962F5A24962FAE245A2E630003
:103F3000220803178C000313210803178E00831631
:103F400003178C170C158B1355308D00AA308D007C
:103F50008C140000FF3EFF3EFF3EFF3EFF3EFF3E53
:103F6000FF3EFF3EFF3EFF3EFF3EFF3EFF3EFF3E69
:103F7000FF3EFF3EFF3EFF3E0C118C1383016400A9
:103F80000D1EBF2F0D1283168101831269080317BE
:103F90008D000313680803178F00DC2783120317B3
:103FA0000C080313A20003170E080313A100080056
:103FB000E90A0319E80A0800831603178C170C1482
:103FC0000000FF3EFF3E8C138301080021081F39CB
:103FD000E8001F3A031968122208E900C627462E96
:103FE00068081E391E3A0319FC2F6808031DFB2FB1
:103FF0006908C039031D8B27D827462EFF3FFF3F96
:104200000200FF00FF00FF00FF00FF00FF00FF00B3
:10421000FF00FF00FF00FF00FF00FF00FF00FF00A6
:10422000FF00FF00FF00FF00FF00FF00FF00FF0096
:10423000FF00FF00FF00FF00FF00FF00FF00FF0086
:10424000FF00FF00FF00FF00FF00FF00FF00FF0076
:10425000FF00FF00FF00FF00FF00FF00FF00FF0066
:10426000FF00FF00FF00FF00FF00FF00FF00FF0056
:10427000FF00FF00FF00FF00FF00FF00FF00FF0046
:10428000FF00FF00FF00FF00FF00FF00FF00FF0036
:10429000FF00FF00FF00FF00FF00FF00FF00FF0026
:1042A000FF00FF00FF00FF00FF00FF00FF00FF0016
:1042B000FF00FF00FF00FF00FF00FF00FF00FF0006
:1042C000FF00FF00FF00FF00FF00FF00FF00FF00F6
:1042D000FF00FF00FF00FF00FF00FF00FF00FF00E6
:1042E000FF00FF00FF00FF00FF00FF00FF00FF00D6
:1042F000FF00FF00FF00FF00FF00FF00FF00FF00C6
:10430000FF00FF00FF00FF00FF00FF00FF00FF00B5
:10431000FF00FF00FF00FF00FF00FF00FF00FF00A5
:10432000FF00FF00FF00FF00FF00FF00FF00FF0095
:10433000FF00FF00FF00FF00FF00FF00FF00FF0085
:10434000FF00FF00FF00FF00FF00FF00FF00FF0075
:10435000FF00FF00FF00FF00FF00FF00FF00FF0065
:10436000FF00FF00FF00FF00FF00FF00FF00FF0055
:10437000FF00FF00FF00FF00FF00FF00FF00FF0045
:10438000FF00FF00FF00FF00FF00FF00FF00FF0035
:10439000FF00FF00FF00FF00FF00FF00FF00FF0025
:1043A000FF00FF00FF00FF00FF00FF00FF00FF0015
:1043B000FF00FF00FF00FF00FF00FF00FF00FF0005
:1043C000FF00FF00FF00FF00FF00FF00FF00FF00F5
:1043D000FF00FF00FF00FF00FF00FF00FF00FF00E5
:1043E000FF00FF00FF00FF00FF00FF00FF00FF00D5
:1043F000FF00FF00FF00FF00FF00FF00FF00FF00C5
:08400000FF3FFF3FFF3FFF3FC0
:00000001FF
